:02000000A32A31
:08000800FF0003088301FE0064
:100010000408FD00B72A0C1E0B28990003141829A8
:1000200083169B0083161C141A089B0A1829AF011B
:10003000AE00FF30AE07031CAF07031C18290330C6
:10004000AB00E53025201928AB01F63EAA00AB092C
:10005000031C3028FE300000AA0703182B28AA072B
:100060000000AB0F2A2800002A1836282A18382842
:1000700008002D0835068039B700AD1F4A28AA09A7
:10008000AB09AC09AD09AA0A0319AB0A0319AC0AFA
:100090000319AD0AB51F5728B209B309B409B50948
:1000A000B20A0319B30A0319B40A0319B50AAE0157
:1000B000AF01B001B101BE01BF01C001C1013508EE
:1000C000340433043204031995282030B600031099
:1000D000AA0DAB0DAC0DAD0DBE0DBF0DC00DC10D0C
:1000E00035084102031D7E2834084002031D7E2886
:1000F00033083F02031D7E2832083E02031C8F286E
:100100003208BE023308031C330FBF023408031C3D
:10011000340FC0023508031C350FC1020314AE0DA5
:10012000AF0DB00DB10DB60B6728B71FA228AE09F1
:10013000AF09B009B109AE0A0319AF0A0319B00A31
:100140000319B10A3E08B2003F08B3004008B400EA
:100150004108B5002E08AA002F08AB003008AC00FB
:100160003108AD001829B301B2011030B6002B0DD3
:10017000B20DB30D2E08B2022F08031C2F0FB302CD
:100180000318C9282E08B2072F0803182F0FB3072A
:100190000310AA0DAB0DB60BB7282A08182920307A
:1001A000B600BE01BF01C001C10103102A1CE62830
:1001B0003208BE0733080318330FBF07340803188B
:1001C000340FC00735080318350FC107C10CC00C28
:1001D000BF0CBE0CAD0CAC0CAB0CAA0CB60BD528EE
:1001E00008001030B900AB01AA01B70CB60C031C13
:1001F000FF282E08AA072F0803182F0FAB07AB0CF8
:10020000AA0CB30CB20CB90BF52832081829AA00B5
:10021000AD1B0C212A081829AA09AB09AC09AD09A4
:10022000AA0A0319AB0A0319AC0A0319AD0A08009C
:100230008313831203130000080026080319A5295D
:10024000220803199D2A23082706C900A317A71708
:10025000C7012308C4002408C2002508C3002908D8
:10026000C3022808031C280FC2022708031C270FFB
:10027000C402C401C201C301031C45290310A30C1D
:10028000A40CA50CC40C0130C7002608A202031C54
:100290004F297E304707A20703188F2A54297E3042
:1002A0004707A207031C842A1830C800C30DC20DDB
:1002B000C40DA50DA40DA30DC70D2908A50228087E
:1002C000031C280FA4022708031C270FA302270DD5
:1002D000C704471C6D29431478292908A507280855
:1002E0000318280FA40727080318270AA307431099
:1002F000C80B5629461B431C9C290310A50DA40DB1
:10030000A30DC70D2908A5022808031C280FA40265
:100310002708031C270FA302270D47040139C30731
:100320000318C20A0319C40A031D9C29C40CC20C79
:10033000C30CA20A03198F2AC91FC4134408A300BF
:100340004208A4004308A5000034C615FF34220863
:10035000C400A2014408031900342308C900A317EC
:100360009E30C402C41F0D2AC409C40A08304402C6
:10037000031CE229C400A20D2508A2002408A50040
:100380002308A400A30108304402031CE229C4008E
:10039000A20D2508A2002408A500A40108304402EB
:1003A000031CE229C400A20D2508A200A501083003
:1003B0004402031CE229C400A20DA2014408031D4B
:1003C0000310EC2944080319EC290310A30CA40C16
:1003D000A50CA20CC40BE529461B221CFA29031C00
:1003E000FA29A20A0319A50A0319A40A0319A30AE0
:1003F000A31B1A2AC91F252AA309A409A509A20912
:10040000A20A0319A50A0319A40A0319A30A252A93
:10041000A301A401A501A201252A4614C61F252A6D
:10042000A301C91FFF30A300A400A500A200C90DAD
:10043000A30C252A4614C61FFF34A301C91FFF3091
:10044000A300A400A500C90DA30C22080800A40164
:10045000A5012208C4002508A2002308A50022083F
:10046000A3009E30A200C901A31F422AC409A50906
:10047000A409A309C40A0319A50A0319A40A0319A4
:10048000A30AC917C7012308031D622A2408A30071
:100490002508A4004408A500C401C7152308031DAE
:1004A000622A2408A3002508A400A501C711471645
:1004B0002308031D622A2408A300A401C7152308EA
:1004C00003199D2A4708A202031D031C842A031056
:1004D000A31B712AC40DA50DA40DA30DA20B682AA0
:1004E000842A461B251C9A2AC41F9A2AA50A031986
:1004F000A40A0319A30A031D9A2AA30CA40CA50C91
:10050000A20A03198F2A9A2A4615C61FFF34013002
:10051000A200A301A401A501C90DA30CFF34C614B8
:10052000C61FFF34FF30A200A300A400A500C90D20
:10053000A30CFF34C91FA3130034A301A401A50118
:10054000C401A201003483160F30990020309800B6
:100550008312803098006030C600A0014B308316B3
:100560008600FF308500073083129F004E2C05184F
:10057000BD2A8316AA018312C32A8518C22A013014
:100580008316AA0083128316AA088312031DD32A96
:10059000CA08031DCE2ACB080319D22ACA034A0A65
:1005A0000319CB03E42A8316230883124B02031C8E
:1005B000E12A031DE42A8316220883124A02031843
:1005C000E42ACA0A0319CB0A8B107D0884007E082E
:1005D0008300FF0E7F0E09008B138B1FF12A8B13F4
:1005E000ED2A8B100B16831601178B178312080048
:1005F0008130831620028312031C102B8030831657
:10060000A0022008003C8312EE000030031CFF3ED5
:10061000EF00F001EF1F0D2BF0037008F100172B16
:10062000F101F001EF01831620088312EE00813002
:10063000831624028312031C2F2B80308316A402FE
:100640002408003C8312F2000030031CFF3EF3003C
:10065000F401F31F2C2BF4037408F500362BF5017D
:10066000F401F301831624088312F20008008316B4
:1006700023088312AB00831622088312AA00AF015D
:100680007830AE00B320E8002B08E9005508AB0035
:100690005408AA006908AF006808AE00B320FA0049
:1006A0007A0810208316A0008312B7017A08B600DA
:1006B0006908AF006808AE00F120F6003308F700C3
:1006C00076085402F8007708031C013E5502F90031
:1006D000FA0A7A0810208316A4008312F8226E0802
:1006E0007202D8007308D9006F08031C6F0FD9027B
:1006F0007408DA007008031C700FDA027508DB005A
:100700007108031C710FDB025B08AD005A08AC00D6
:100710005908AB005808AA00B501B4017908B30024
:100720007808B200CF202D08A5002C08A4002B08C3
:10073000A3002A08A20029222508BD002408BC0025
:100740002308BB002208BA006908A3006808A200B9
:1007500027222508A9002408A8002308A7002208AA
:10076000A6003D08A5003C08A4003B08A3003A08E9
:10077000A2001D212508E7002408E6002308E50063
:100780002208E4006708A5006608A4006508A30025
:100790006408A200A7212308ED002408EC00250826
:1007A000EB002208EA0054086E07BA006F08BB008D
:1007B00055080318550FBB077008BC00003003181C
:1007C0000130BC077108BD00003003180130BD07BF
:1007D0003A086A07D4003B080318013E6B07D500AE
:1007E0000800AD01AC015508AB005408AA00B501E2
:1007F000B4010230B300B201CF202D08BD002C0897
:10080000BC002B08BB002A08BA003D08AD003C081C
:10081000AC003B08AB003A08AA00B501B40183164E
:1008200026088312B300831625088312B200CF2056
:100830002D08DB002C08DA002B08D9002A08D80084
:100840005B08AD005A08AC005908AB005808AA0074
:10085000B501B401B3012D30B20039202D08DB0001
:100860002C08DA002B08D9002A08D8005B08AD0054
:100870005A08AC005908AB005808AA00B501B401E9
:10088000831623088312B300831622088312B20052
:1008900039202B08D5002A08D40008000330AF0007
:1008A000E8301820861201308316A1008312CB0194
:1008B000CA017B3010208316A7008312AD01AC0162
:1008C0000230AB00AA01B501B401B30183162708B9
:1008D0008312B200CF202D08BD002C08BC002B08CD
:1008E000BB002A08BA003D08AD003C08AC003B083C
:1008F000AB003A08AA00B501B401B3012D30B20033
:1009000039202D08D3002C08D2002B08D1002A084A
:10091000D00051088316A900831250088316A8003E
:100920007E30831210208316A200831212208316B9
:10093000A3007C30831210208316A500831212209E
:100940008316A6008312EC220519A82CCB01CA013C
:100950008B1FAC2C8B13A82C4B08D5004A08D40055
:100960008B173723F1238618E22C5508B30054085F
:10097000B200B401B501003ECC00F030CD00330828
:100980000318330FCD07FF30CE0034080318340F9F
:10099000CE07FF30CF0035080318350FCF074F08BB
:1009A000AD004E08AC004D08AB004C080721CC0050
:1009B0002B08CD002C08CE002D08CF004D08D50007
:1009C0004C08D4008519FA2C831628088312D40702
:1009D000831629080318013E8312D50710305502EB
:1009E000031CFA2C031DF82C01305402031CFA2CB2
:1009F0001030D502061B1B2D061641305407BA00D5
:100A000055080318013EBB008316210883123A07DC
:100A1000D6003B080318013ED70041300B20540894
:100A20000B2055080B208316210883120B20560833
:100A30000B2057080B20061B1E2D1B2D0612A42C65
:040A40006300202D02
:02400E00223F4F
:1042000000000000000001000100010001000200A8
:104210000200020003000300030003000400040086
:104220000400050005000500050006000600060064
:104230000700070007000700080008000800090041
:104240000900090009000A000A000A000B000B001F
:104250000B000B000C000C000C000D000D000D00FD
:104260000D000E000E000E000F000F000F000F00DB
:1042700010001000100011001100110011001200B8
:104280001200120013001300130013001400140096
:104290001400150015001500150016001600160074
:1042A0001700170017001700180018001800190051
:1042B0001900190019001A001A001A001B001B002F
:1042C0001B001B001C001C001C001C001D001D000E
:1042D0001D001E001E001E001F001F001F001F00EB
:1042E00020002000200021002100210021002200C8
:1042F0002200000000005A00670000009000060045
:00000001FF
